:020000001028C6
:08000800080082077E34303449
:080010006D34793433345B34A4
:080018005F3470347F347B3447
:080020001C306500FF30660092
:080028000510851400308A0068
:080030000030A300A400A100B0
:08003800A2009F00A000A70038
:08004000A900A5000130A60093
:08004800A8000930AB000530EF
:08005000AA0085102B280430E2
:080058008D0008308C008C0BB8
:080060002F2885140000851013
:0800680000008D0B2D2808306B
:080070008C008C0B3928000004
:08007800851400008510000052
:0800800085140430251803303B
:080088008D0008308C008C0B88
:080090004728851000008514CB
:0800980000008D0B452800005B
:0800A00008308C008C0B522883
:0800A80085101E3008218510AF
:0800B000072185144E30970072
:0800B8000E3098007E30990023
:0800C0004E309A0037309B001E
:0800C80067309C0030309D0000
:0800D0004E309E000D308C0043
:0800D8008C0B6C286F288510C9
:0800E0001E21851010300821DB
:0800E80085100721851427088B
:0800F0000520970026080520F9
:0800F800980025309900290849
:0801000005209A0028080520E3
:080108009B0025309C002B0830
:0801100005209D002A080520CE
:080118009E00052185101E2147
:08012000851010300821851044
:080128000721851420080520C1
:0801300097001F08052098004C
:080138000130990022080520A6
:080140009A00210805209B0034
:0801480000309C002408052092
:080150009D00230805209E001C
:08015800052185101E21851010
:08016000A50ACE30250700308E
:0801680085140318A50003181B
:08017000A30AF630230700305A
:080178000318A3000318A40AF8
:08018000FA30240700300318D7
:08018800A4000318A10AF630DF
:08019000210700300318A10053
:080198000318A20AFA30220745
:0801A00000300318A20003184F
:0801A8009F0AF6301F0700302A
:0801B00003189F000318A00AC8
:0801B8001F0820180A3EA018E0
:0801C000143EE83E0030031874
:0801C8009F000318A0000318BA
:0801D000A60A052185103B3051
:0801D8000821851000008514C8
:0801E0000430251C05308D00E0
:0801E80008308C008C0BF62896
:0801F0008510000085140000D9
:0801F8008D0BF42807308C0088
:080200008C0B002903292928B9
:080208000000000000000800E6
:08021000FF3E85148D000C294E
:0802180011308C008C0B0E2943
:080220000000122985100721DE
:0802280085148D0B0C29000068
:0802300011308C008C0B1A291F
:080238000000080010308400F2
:080240008514003096009500C2
:08024800940093009200910064
:08025000900006308C008C0BBD
:080258002B292E29CD21851070
:0802600007218514CD21CD21F9
:08026800851007218514CD214A
:08027000CD2185100721851442
:08027800CD21CD218510AE213E
:080280008510AE218510AE21AE
:080288008510AE218510AE21A6
:080290008510AE218510AE219E
:080298008510AE218510BD2187
:0802A0008510BD218510BD2170
:0802A8008510BD218510BD2168
:0802B0008510BD218510BD2160
:0802B8008510BD218510BD2158
:0802C0008510BD218510BD2150
:0802C8008510BD218510BD2148
:0802D0008510BD218510BD2140
:0802D8008510BD218510B32142
:0802E0008510B3218510B32144
:0802E8008510B3218510B3213C
:0802F0008510B3218510B32134
:0802F8008510B3218510C5211A
:080300008510C5218510C521FF
:080308008510C5218510C521F7
:080310008510C5218510C521EF
:080318008510C5218510C521E7
:080320008510C5218510C521DF
:080328008510C5218510C521D7
:080330008510C5218510C521CF
:080338008510C5218510B821D4
:080340008510B8218510B821D9
:080348008510B8218510B821D1
:080350008510B8218510B821C9
:080358008510B82916088E007B
:0803600085140621E7291008AD
:080368008E0085140621E7292F
:0803700013088E00851406211C
:08037800E72911088E0085142D
:0803800015088F00C3290000DD
:08038800112A12088E008514F1
:0803900014088F00CB290000C6
:08039800112A171800141818AF
:0803A0008014191800151A1849
:0803A80080151B1800161C183B
:0803B00080161D1800171E182D
:0803B8008017970C980C990CBA
:0803C0009A0C9B0C9C0C9D0C97
:0803C8009E0C840A08000E18C7
:0803D0000514EA2900000510E4
:0803D8008E180514EF29000046
:0803E00005100E190514F429A3
:0803E800000005108E19051438
:0803F000F929000005100E1AA6
:0803F8000514FE2900000510A8
:080400008E1A0514032A000006
:0804080005100E1B0514082A63
:08041000000005108E1B05140D
:080418000D2A00000510000090
:0804200008000E180514051078
:080428000F18051405108E18D1
:08043000051405108F180514D6
:0804380005100E190514051052
:080440000F19051405108E19B7
:08044800051405108F190514BD
:0804500005100E1A0514051039
:080458000F1A051405108E1A9D
:08046000051405108F1A0514A4
:0804680005100E1B0514051020
:080470000F1B051405108E1B83
:08047800051405108F1B05148B
:0604800005100000080059
:02400E00190097
:00000001FF
